:10000000C828A0008417800484138E010C1C8E0065
:1000100023200319C32823200319C3282320C3281E
:10002000A00059200C080D040319C328BD20841317
:100030002008800664001C281D288C0A03198D0FD7
:100040001A288006C32820088E0601308C008D01F6
:10005000000820050E06031D08008C0A03198D0FE9
:10006000282808008F002208840020095A208413C1
:100070008F080319C328F03091000E0880389000D3
:10008000F03091030319910003198F030319C3285A
:1000900049285D2003010C1820088E1F20088E08B7
:1000A00003190301900F562880063D2857280000A9
:1000B0004028FF3A84178005C3280D080C04031953
:1000C0008C0A80300C1A8D060C198D068C188D0642
:1000D0000D0D8C0D8D0DC3288F018E00FF308E0706
:1000E000031C8F07031CC32803308D00DF307A20E8
:1000F0006E288D01E83E8C008D09FC30031C83289E
:100100008C07031880288C0764008D0F80280C183A
:1001100089288C1C8D2800008D2808008E00033053
:10012000912894000F080D02031D98280E080C0258
:10013000043003180130031902301405031DFF3089
:10014000C32891019001103092000D0D900D910D7A
:100150000E0890020F08031C0F0F91020318B72816
:100160000E0890070F0803180F0F910703108C0D4E
:100170008D0D920BA5280C08C3288C098D098C0ABB
:1001800003198D0A08008313031383126400080007
:100190008316850108308600831206118316061126
:1001A000831206108316061083128610831686109B
:1001B00083120130AC00640006302C020318E328DF
:1001C0007721AC0FDB289C2124088C0025088D00AA
:1001D0008F0107308E20031DF7280130AC0064002A
:1001E00006302C020318F7285221AC0FEF289C216F
:1001F00024088C0025088D008F0107308E20031DF8
:100200000B290130AC00640006302C0203180B29C6
:100210005221AC0F03290130AC00640006302C02DF
:10022000031815291821AC0F0D29D92863001629A8
:10023000AA30A900BB21A030A800A030AA00BB2191
:100240006430A900BB217830A8007830AA00BB2117
:1002500008000630A2001030A0005A308E00013095
:10026000322050308E00023032207D308E0001303E
:1002700032205A308E000230322064308E0002303C
:100280003220AA30A900BB217830A8007830AA001B
:10029000BB216430A900BB21A030A800A030AA0077
:1002A000BB2108000630A2001030A0008C308E0068
:1002B0000130322050308E00023032207D308E00EE
:1002C000013032205F308E0002303220AA30A90087
:1002D000BB217830A800A030AA00BB216430A9005F
:1002E000BB21A030A8007830AA00BB21080006304E
:1002F000A2001030A0008C308E0001303220783007
:100300008E00023032206E308E0001303220643098
:100310008E0002303220AA30A900BB21A030A800F4
:100320007830AA00BB216430A900BB217830A80036
:10033000A030AA00BB21080001308C008D010630DE
:1003400084000430102001308C0006308400083016
:1003500001200C08A6000D08A70026088C0027081D
:100360008D000F308E008F01A120A4000D08A50084
:1003700001306C2008000130AB0064000B302B0210
:100380000318DB2929088C008D0106308400803099
:10039000102028088C008D01063084004030102089
:1003A0002A088C008D0106308400203010200D308A
:0803B0006C20AB0FBD29080011
:02400E00F53F7C
:00000001FF
